:1000000000308A001D2C00000A108A100A11820795
:100010004C343A342034253455342034203452348E
:100020003A34203425345534003400347830840098
:10003000FC308005800C800C00080319232821283F
:100040000000800B202800347508F7007408F600C3
:10005000F608031D2E28F708031949288316861170
:100060008312861583160611831206117208F80092
:100070001620831606118312061583168611831225
:1000800086117208F800162076080319F703F603A4
:100090002828003473308400000803195E280130DA
:1000A000A100A001A00B5228A10B51284A30A000AA
:1000B000A00B582800000000800B4F2800346B086C
:1000C000840075088000840A8001EB0A00347608F9
:1000D000A101750203186F287508A0007B28A001F4
:1000E0000830F700F50DA00D760820020318A000D7
:1000F000A10DF70B7228003421087308F500643055
:10010000F60067202008F30021083030031D8F28F7
:100110007418F415F4199528741A20309128F411E4
:100120007412A1072108F5005F207308F5000A305A
:10013000F60067202008F30021083030031DA428B2
:10014000F419A828741A2030A1072108F5005F20AF
:100150003030F3077308F5005F200034B801351C18
:10016000B3283510B42835140034351CE828BC11E8
:100170003C0883168700831287154930A000A00B26
:10018000BF2800000000BC113C08831687008312C2
:1001900087114930A000A00BCB2800000000BC1143
:1001A0003C0883168700831287154930A000A00BF6
:1001B000D72800000000BC113C088316870083127A
:1001C00087111930A000A00BE32800000000FE28D2
:1001D000BC113C0883168700831287158930A00064
:1001E000A00BF028BC113C088316870083128711EE
:1001F0007230A000A00BFA28000000000034F501C6
:100200007508073C031C492974080139F600BA082F
:1002100003190C2900300D290130F700B908031922
:1002200013290030142901307705003A03192729D2
:100230007608F7000310B70CB60C030801397706EF
:10024000013C031D27298430B7060830B606F6089E
:10025000031D2C29AE204429B908031D3029B80AF2
:10026000B90803193529003036290130F70038085C
:10027000053C03193D2900303E2901307705003A3D
:1002800003194429B520AE20B5200310F40CF50A5B
:1002900000290034831606148312061C752A0130C7
:1002A000EF00F430EE006F08033C031C6B29031DC4
:1002B0005D296E081F3C031C6B296F08F3006E0854
:1002C000F2006F08F5006E08F40024206430EE0799
:1002D0000318EF0A53290430F200FA30F3004A20E1
:1002E000F20B6D29831606138312061383168613E9
:1002F0008312861383160612831206128316861241
:1003000083128612831686128312861283160612B1
:10031000831206160430F200FA30F3004A20F20B82
:100320008C298316061283120612831686128312F4
:1003300086120430F200FA30F3004A20F20B9B29B7
:1003400083160612831206128316861283128616ED
:100350000430F200FA30F3004A20F20BAA29831687
:100360000612831206128316861283128612043036
:10037000F200FA30F3004A20F20BB9290330F300FF
:100380007030F200F5016430F40024200430F200F3
:10039000FA30F3004A20F20BC82983168613831221
:1003A000861383160613831206170430F200FA3000
:1003B000F3004A20F20BD729831606138312061383
:1003C00083168613831286130430F200FA30F3008A
:1003D0004A20F20BE62983160613831206138316AE
:1003E0008613831286170430F200FA30F3004A2095
:1003F000F20BF52983160613831206138316861350
:10040000831286130430F200FA30F3004A20F20B14
:10041000042A0330F3007030F200F5016430F40078
:1004200024200430F200FA30F3004A20F20B132AA1
:1004300083168613831286138316061383120617F8
:1004400083168612831286128316061283120616EC
:100450000430F200FA30F3004A20F20B2A2A831605
:1004600006138312061383168613831286138316CC
:100470000612831206128316861283128612043025
:10048000F200FA30F3004A20F20B412A83160613D9
:100490008312061383168613831286178316061299
:1004A0008312061283168612831286160430F20017
:1004B000FA30F3004A20F20B582A831606138312EF
:1004C000061383168613831286138316061283126D
:1004D000061283168612831286120430F200FA3056
:1004E000F3004A20F20B6F2A4A29831686148312DE
:1004F000861C192B3C163C08831687008312071AAA
:100500008D2A0430F3004C30F200F5016430F40021
:1005100024203230F3004A207A2A0830A1001F0834
:10052000C73921049F000630A000A00B952A0000C7
:100530001F151F19992A1E08F1000030A1001F087D
:10054000C73921049F000630A000A00BA52A000097
:100550001F151F19A92A1E08F0003D30EB004C3072
:10056000F5005F203A30F5005F202030F5005F2075
:100570007008F3001830F4007C200530F200720897
:100580000420F20AF5005F200A307202031DBF2A20
:100590007108F3001830F4007C203D30F200351073
:1005A000FF30B700B600B8010130B900BA01BB0195
:1005B0003B08093C031CE12A7E30F400FF20BB0A03
:1005C000D82AB901BB013B080F3C031CF02A253097
:1005D0003B0784000008F300F400FF20BB0AE32A75
:1005E000BB01720884000008003A0319002B72084E
:1005F00084000008F300F400FF20F20ABB0AF12A8D
:100600000130BA00FF30B606B7063608F400FF2006
:100610003708F400FF20BA010130B9007E30F40041
:10062000FF200430F200FA30F3004A20F20B132BC3
:10063000752A8A115E2C83160613831206138316FD
:1006400086138312861783160612831206128316E8
:100650008612831286160230EE009630F3004A208E
:10066000EE0B2D2B831606128312061283168612AA
:1006700083128612831606138312061383168613BB
:10068000831286130330F300E830F2000330F500E4
:10069000E830F40024200230EE00FA30F3004A2063
:1006A000EE0B4D2B0330F300E830F2000330F50081
:1006B000E830F40024200430EE00FA30F3004A2041
:1006C000EE0B5D2B8A118A2C01306702FD3E031868
:1006D000A42B033E102C83168613831286138316D5
:1006E0000613831206178316061283120612831648
:1006F0008612831286160130E700A42B8316861219
:1007000083128612831606128312061683160613A8
:100710008312061383168613831286170230E700AE
:10072000A42B831686128312861283160612831256
:100730000616831606138312061383168613831276
:1007400086170230E700A42B0030A1001F08C7392C
:1007500021049F000330A000A00BAC2B1F151F1914
:10076000AF2B1E0865020318FC2B6E08323C031DDC
:10077000F72B831606128312061283168612831233
:1007800086128316061383120613831686138312AA
:100790008613EE0101306702FE3E0318F72B023E7E
:1007A000172C83168613831286138316061383125F
:1007B00006178316061283120612831686128312F8
:1007C00086160130E700F72B8316861283128612F5
:1007D0008316061283120616831606138312061357
:1007E00083168613831286170230E700F72B053035
:1007F000F3004A20EE0AAE2B83160613831206136B
:10080000831686138312861383160612831206122A
:1008100083168612831286120330E8008A11102E86
:100820000A108A100A1582077E2B6B2B912B0A1057
:100830008A100A158207E42BD12B84011F3083050F
:10084000073083169F0082308312A5009830A600DF
:10085000A7004030A800A900AA006030AB00863095
:10086000AC00B430AD006030AE00A430AF00B000DA
:10087000B1006130B2000330B300F030B400FF309B
:10088000BC00EB018316061383120613831686132E
:10089000831286138316061283120612831686129B
:1008A00083128612043083169F0083121F08383982
:1008B00001389F008316811783124A290330F30001
:1008C000E830F200F501C830F40024203230F300A3
:1008D0004A200330F300E830F200F501C830F4009C
:1008E00024200430EE00FA30F3004A20EE0B732C83
:1008F0005030E600E5000330E700E800EA01E901D6
:10090000ED01EC013C163C08831687008312071AA0
:100910008A2C1B2BE8010830A1001F08C7392104CD
:100920009F000330A000A00B932C1F151F19962CBD
:100930001E0866020319A22C031CA22CEA01E9017D
:100940000130E8000030A1001F08C73921049F00D2
:100950000330A000A00BAA2C1F151F19AD2C1E08D8
:1009600065020319B82C031CB82CEA01E901E8144C
:100970006808A000033020020319C72C02302002AF
:100980000319DA2C013020020319ED2C002D8316F7
:100990008612831286128316061283120616831697
:1009A00086138312861383160613831206170330E9
:1009B000E700822C83160613831206138316861310
:1009C00083128613831686128312861283160612EA
:1009D000831206160230E700822C83160612831259
:1009E00006128316861283128612831686138312CA
:1009F000861383160613831206170130E700822C34
:100A0000690B4A2DEA08031D4A2DED01EC01013066
:100A10006802FE3E03184A2D023E172E8316061367
:100A20008312061383168613831286176430F3002D
:100A30004A20831606138312061383168613831225
:100A40008613831686128312861283160612831269
:100A500006160230E7004A2D83160612831206128C
:100A600083168612831286166430F3004A2083169A
:100A700006128312061283168612831286128316BA
:100A8000861383128613831606138312061701300A
:100A9000E7004A2D6908183C031D122E6A08153C10
:100AA000031D122E0330F3002030F2000130F50058
:100AB000F430F40024203230F3004A200330F300F5
:100AC0002030F2000130F500F430F4002420013031
:100AD0006702FD3E0318E62D033E1D2E8316061306
:100AE0008312061383168613831286138316061247
:100AF000831206128316861283128612831606123A
:100B00008312061283168612831286160830EE00B0
:100B1000C830F3004A20EE0B882D8316061283128C
:100B200006128316861283128612E62D831606138A
:100B300083120613831686138312861383160612F6
:100B400083120612831686128312861283160613E8
:100B50008312061383168613831286170830EE005D
:100B6000C830F3004A20EE0BB02D83160613831213
:100B700006138316861383128613E62D8316061337
:100B800083120613831686138312861783160612A2
:100B90008312061283168612831286160830EE0020
:100BA000C830F3004A20EE0BD02D831606138312B3
:100BB0000613831686138312861383160612831276
:100BC00006128316861283128612E62D831686126B
:100BD0008312861283160612831206168316861354
:100BE0008312861383160613831206170230EE0053
:100BF000C830F3004A20EE0BF82D8316061383123B
:100C00000613831686138312861383160612831225
:100C1000061283168612831286120330E700642BB5
:100C2000EA01E901E90A0319EA0A822C63000A10C1
:100C30008A140A1582072C2D0E2D0A108A140A1503
:080C40008207962D6E2DBE2DDA
:02400E00793FF8
:00000001FF
